:020000020000FC
:1000000012C063C07FC0189518951895189518955B
:100010001895189518951895189518951895189578
:100020004FC018951895002404E0102E08E0202EEB
:1000300009E0302E00E2402E03E7602E00E7702E2C
:1000400001E6802E0EE6902E0DE0502E04E00EBF4D
:100050000FE50DBFD1E0C0E0B1E0A0E0112707E05F
:1000600005BF00EC0BBF08E1A89501BD00E101BD93
:10007000002700BD05E009B900E40BB908E00AB9A2
:1000800006E800BD04E000BF08E408B903E50D93ED
:1000900004E70D9301E60D9302E70D9304E70D933A
:1000A0000DE00D9378945D9BFECFDB130010CA1317
:1000B0000010F9CF09910CB9D1110010D1E0F3CFA4
:1000C00019E6459B10521D9335C0110F8399139566
:1000D0002395231100100FC02111001002C022111E
:1000E00018951A3020F0195C1D93112723C0105D5C
:1000F0001D9311271FC010FF8D9210FD9D92222786
:10010000112718C0829B1895839904C022271127B4
:100110006D9210C0222711277D92B1110010B1E01D
:10012000CA1306C0DB1304C01197B0110010B3E06E
:100130005D9200C0B1110010B1E0CA131895DB1335
:0C01400018951197B0110010B3E018954D
:00000001FF
